:020000040000FA
:020000004D2889
:080008000900170892009301A2
:10001000130B0828120B07280034003086008316C3
:1000200086018312140886001508850085010301E6
:1000300086008316FF308600831200348316FF305B
:1000400086008312150885000000060894008501CB
:100050000034043095001E3094000D20052000303F
:1000600094000D200520103094000D200520003054
:1000700094000D20052090111016100894000D20FA
:100080000520003094000D2005201F3094000D2025
:100090000520003094000D200034FF30970005202B
:1000A00005208B0183168730810083120030850084
:1000B000831618308500831208308C008D018E0164
:1000C0008F0194019601043095000D2003019400E6
:1000D000073095000D20053095000D20013094006B
:1000E000063095000D20033095000D208F01003063
:1000F00095001E201408031DBA28013095001E200B
:100100001408031DF428023095001E201408F0394D
:100110009100110C110C110C110C11089000140815
:100120000F39031D0D298E109101110B95280E1A00
:100130009F2803019400043095000D200E16901D99
:10014000B7288519B7280E18AA280E140130810087
:100150000A3096000108031D7628010A160B76283E
:100160008E1976289030970029208E1576288E11CA
:100170000E1076288F0090300F0203196729813006
:100180000F02031DC6281A308D00302982300F025D
:10019000031DCD281B308D00302984300F02031D34
:1001A000D4281C308D00302988300F02031DDB2835
:1001B0001D308D00302911300F188D0014308F182C
:1001C0008D0017300F198D001E308F198D000130F2
:1001D0000F1A8C0002308F1A8C0004300F1B8C0019
:1001E00008308F1B8C001A298F0012300F188D00D9
:1001F00015308F188D0018300F198D0010308F19A1
:100200008D0010300F1A8C0020308F1A8C00403077
:100210000F1B8C008F1B0E151A298F0013300F181F
:100220008D0016308F188D0019300F198D001F307A
:100230008F198D008E1865298E140E1D242990307B
:10024000970029200E1165290F080F390319652918
:100250008C1D3E290D089400043095000D20652961
:100260008C1D3E290D089400043095000D200030AF
:1002700095001E201408031D372965290D03073931
:1002800094000C1C4929073095000D20053095007D
:100290000D208C1C4E29053095000D200C1D532976
:1002A000073095000D200C1E5B29063095000D20AF
:1002B000033095000D208C1E6029033095000D2021
:1002C0000C1F6529063095000D200E1276288E161B
:1002D000FF309700980118089400053095000D2014
:1002E000073095000D200E309400043095000D204D
:1002F000052000309400043095000D2005200520D5
:100300000520052018089400033095000D200630C4
:1003100095000D2029309400043095000D20052013
:1003200000309400043095000D20052005200520A4
:100330000520013095001E20903014020319A429D5
:10034000180A073018056B290A3091008030970091
:1003500008309400043095000D20052000309400F2
:10036000043095000D2005200830940004309500DD
:100370000D20052000309400043095000D20110B55
:10038000A8298E129401950103014D28283043308D
:1003900029304730573036304230573058302E30C1
:0203A000033028
:02400E00F93F78
:00000001FF
